:1000000000298A0182002F345634323450340034AF
:100010008A012B08AB0A82002F340F3400344D3490
:1000200012340034313415340034543431295A3404
:0E003000432956342E290D342429003400347F
:100200008316B630900014308500831207309900B1
:100210002430E3216400051A0A29C6210C30AB0002
:10022000DB21AC000820003A03191E292C06031913
:100230001B29AB0A12290820AB0010290820003A1C
:10024000031D0A293F30E321682227210A290D30A6
:10025000E32915300F292E30E32129297830AF21E9
:1002600029299921AA002A08A03C031C2229DB2164
:10027000A1000D3A03192429A11721084E212A08AB
:100280004E21AA0A3329AA01A0304E212A084E2164
:10029000AA0A2A08A03A031D44292429A2000830EA
:1002A000A60005195129051D5329221C8510221865
:1002B0008514A20C0830A700A70B5C29A60B5529B2
:1002C00085100800AD000230D2000A304D222D0802
:1002D0006F21201908002721D20B672908007221FD
:1002E0007D210800D1005108D10A0120A100003A67
:1002F000031908002108E3217329AF01201164309C
:10030000AE0058220222A10020188929AE0B8129B3
:1003100008002F080A3A03197D292F08303E84006F
:1003200021088000AF0A0D3A031D7F29AF01201577
:100330000800A201DB21A1003030A102031CAD297D
:100340000A3021020318AD290310A20D2208A20DC4
:10035000A20DA2072108A2079A2922080800A011CD
:10036000D3006430B7210A30B721A0150130D50081
:100370003030D4005508D302031CC129D40AA0157B
:10038000BB29D3075408A019E3210800AF010222BA
:10039000201CC7296400A1002F081C3A03190A2950
:1003A00030302F07AF0A8400210880000D3A031D6A
:1003B000C729AF01080030302F07AF0A84000008BA
:1003C0000800AF030800A20002304D228316051278
:1003D00083120430FA210230FA210830A6000130DD
:1003E000A20D03180330FA21A60BEF298316051678
:1003F00083120800A100582205125822A10BFD29E2
:1004000005160800A0102010051A08001A221A224A
:10041000D9000830A600A2011A220319182AA10047
:100420005908A102A20DA60B0C2A220820140800CC
:10043000A0140800A101A10A03190800000000008F
:1004400000000000000000000000000000000000AC
:10045000000000000000000000000000051A1B2A38
:10046000A101A10A0319080000000000000000001B
:10047000000000000000000000000000000000007C
:100480000000000000002108051E312A0800DD00E0
:1004900064304D22DD0B482A0800DC005C22DC0BB6
:1004A0004E2A080001305D2A02305D2A05305D2A9F
:1004B0000A305D2A32305D2A6430DB000000000023
:1004C00000000E30DA00DA0B632ADB0B5E2A08002C
:1004D0005608D7075708D8075808D60ED607080079
:1004E0002012D000CF00CE00051E2016CE0B742A9D
:0A04F000CF0B732AD00B722A08000C
:02400E00A3010C
:00000001FF
